:100000000C9470000C9498000C9498000C94980038
:100010000C9498000C9498000C9498000C94980000
:100020000C9498000C9498000C9498000C949800F0
:100030000C9498000C9498000C9498000C949800E0
:100040000C942B0A0C9498000C94F8070C94D2078B
:100050000C9498000C9498000C9498000C949800C0
:100060000C9498000C94980057726974696E67201C
:100070002800646573657269616C697A654A736F9B
:100080006E2829206661696C65643A2000000000D2
:100090000800020100000304070000000000000047
:1000A0000000000000250028002B000000000024B4
:1000B0000027002A000404040404040404020202C9
:1000C0000202020303030303030102040810204099
:1000D0008001020408102001020408102000BE0D57
:1000E00011241FBECFEFD8E0DEBFCDBF23E0A4E9CF
:1000F000B2E001C01D92A936B207E1F712E0A0E01C
:10010000B1E0E6E9F1E202C005900D92A439B10731
:10011000D9F710E0C0E7D0E004C02197FE010E94AB
:10012000590FCF36D107C9F70E94750A0C94C91030
:100130000C940000FC01918D828D981761F0828DE6
:10014000DF01A80FB11D5D968C91928D9F5F9F730B
:10015000928F90E008958FEF9FEF0895FC01918DAD
:10016000828D981731F0828DE80FF11D858D90E01A
:1001700008958FEF9FEF0895FC01918D228D892FB7
:1001800090E0805C9F4F821B91098F73992708959F
:1001900080E090E0892B29F00E94570781110C9490
:1001A000000008954F925F926F927F928F929F927C
:1001B000AF92BF92DF92EF92FF920F931F93CF9374
:1001C000DF938C01EB0188818B3231F08D3229F481
:1001D0002196EE24E39402C02196E12C888190EDD3
:1001E000980F9A3018F08E3209F0D4C060E070E0B9
:1001F000CB01FE012191A0ED8A2E820E39E0381547
:1002000008F16A3929E97207820729E19207E0F4C7
:10021000AAE0B0E09B01AC010E941D0F912CA12C23
:10022000B12C24013501409450946094709446168A
:1002300057066806790640F0680D791D8A1D9B1DDA
:10024000EF01D7CF222339F0F12CEAE08E2E912C4A
:10025000A12CB12C13C0F801608371838283938336
:100260000E94FE0DF8016483758386839783EE20D8
:1002700011F08AE001C088E0F801D7C0611571056E
:10028000F0E88F07910540F0A50194010E94370F17
:10029000CA01B901F394F2CFFE01299130ED320F7A
:1002A0003A3010F4F394F8CF2E32F1F4EF012196A6
:1002B000FE012196208150EDD52ED20E29E02D157C
:1002C00098F06C3C3CEC73073CE08307910580F7A9
:1002D000AAE0B0E09B01AC010E941D0F6D0D711DE5
:1002E000811D911DFA94E4CF20812F7D253409F0E2
:1002F0004CC021812D3221F43296BB24B39406C028
:100300002B3211F0319601C03296B12CDF01C0E0E2
:10031000D0E04AE0A42E2F2D0F2C000C330BFD0152
:10032000DD9040ED4D0D4A3050F5AC9EA001AD9EE4
:10033000500D1124CD2DDD0CDD0BE097C40FD51F22
:10034000A9014C0F5D1F473251054CF3BB2059F0FA
:10035000EE2029F080E090E0A0E0B0E860C080E00E
:1003600090E0DC015CC0E11005C080E090E0A0E816
:10037000BFE755C080E090E0A0E8BFEF50C0BB20D1
:1003800031F0D195C195D10902C0C0E0D0E0208103
:10039000222359F0F80110821182128213821482F2
:1003A000158216821782108641C0CF0DD11DF7FC31
:1003B000DA950E94FE0D1C161D06ACF4F12CC0FF50
:1003C0000CC024E0F29EF0011124E25EFE4F208179
:1003D0003181428153810E945F0ED595C795F39478
:1003E000209769F718C0D195C195D109F12C2097B4
:1003F00091F0C0FF0CC024E0F29EF0011124EA5FEE
:10040000FE4F20813181428153810E945F0ED5953C
:10041000C795F394ECCFDC01CB01E110B058F801A3
:1004200084839583A683B7838CE08087C801DF919E
:10043000CF911F910F91FF90EF90DF90BF90AF9001
:100440009F908F907F906F905F904F900895982F1E
:1004500080ED890F8A3020F081EA890F8C3110F409
:1004600081E008958FEB890F8A31D0F39B32C1F37D
:1004700081E09D3221F09E3219F080E008950895C8
:100480000895FC01808581110AC0A281B381CD014C
:100490000196938382838C91878381E08087878113
:1004A0000895DF92EF92FF920F931F93CF93DF9304
:1004B000EC017B010C811D810E944102D82E18861F
:1004C000CE010E9441021886D81659F1811103C04D
:1004D00081E090E037C08C35D9F4CE010E94410212
:1004E0008823B1F3853719F0E2E6F1E006C084E035
:1004F00090E028C0891729F0329690819111FACFA7
:1005000006C08181811103C082E090E01BC0188683
:10051000EC81FD819F012F5F3F4F3D832C838083C2
:10052000CFCFEC81FD81CF0101969D838C8310821A
:10053000F70111830083012B19F483E090E002C0DE
:1005400080E090E0DF91CF911F910F91FF90EF90AD
:10055000DF9008951F93CF93DF93EC01CE010E94AB
:1005600041028B302CF489300CF58823C1F032C065
:100570008032E1F08F3219F08D3061F517C01886A6
:10058000CE010E9441028A3219F08F32C9F01FC099
:10059000188610E0CE010E944102811103C081E063
:1005A00090E01AC08F3221F4112311F01886D6CFB3
:1005B00011E08A3209F010E01886ECCF8A3071F22F
:1005C0001886CE010E9441028111F8CFE8CF82E067
:1005D00090E002C080E090E0DF91CF911F910895FC
:1005E000CF93DF93DC01EB01EC81FD818A819B815C
:1005F0000896E817F90718F480E090E021C03897D2
:10060000FD83EC833097C1F31296CD91DC91139763
:10061000209751F0CF018C1B9D0B23E0959587957A
:100620002A95E1F78D8303C01196FC93EE93139600
:10063000FC93EE9312971582148217821682CF01D3
:10064000DF91CF910895562FB901242F452FFC013A
:10065000828193810E946B0981E00895FC01848D61
:10066000DF01A80FB11DA35ABF4F2C91848D90E0DC
:1006700001968F739927848FA689B7892C93A089B7
:10068000B1898C91837080648C93938D848D981341
:1006900006C00288F389E02D80818F7D80830895D4
:1006A000CF92DF92EF92FF92CF93DF93CDB7DEB779
:1006B00029970FB6F894DEBF0FBECDBFFC01892B82
:1006C00009F45FC094819F77963059F018F4943004
:1006D00090F457C09A3051F09C30A9F1983009F04D
:1006E00050C080819181A281B38121C0808191819C
:1006F000A281B38112C060817181CE0101960E94F6
:10070000D20089819A81AB81BC8129852A3029F068
:100710002C30A1F02830A9F50AC0813020E89207DA
:10072000A105B10570F59195819591092CC08115B0
:1007300020E89207A105B10530F123C0CD80DE800D
:10074000EF80F88404C0C080D180E280F38020E094
:1007500030E040E057ECC701B6010E94950F87FDDD
:1007600010C020E03EEF4FEF56E4C701B6010E94F3
:10077000F90D181634F0C701B6010E945F0FCB01C6
:1007800002C080E090E029960FB6F894DEBF0FBE5D
:10079000CDBFDF91CF91FF90EF90DF90CF90089584
:1007A0000F931F93CF93DF93FC01248125FF20C07B
:1007B0008B01C081D1812097D9F06E817F81601734
:1007C0007107A1F00115110541F06115710529F0BE
:1007D000C8010E94C010882349F08D81882341F010
:1007E000F8E08F02C00DD11D1124E5CFCE0102C06B
:1007F00080E090E0DF91CF911F910F910895FC016F
:10080000892BE1F084818F77883019F08A3061F08C
:1008100015C081E04081518162817381411550484A
:100820006105710560F00AC081E0408151816281FB
:100830007381413050486105710508F080E00895EA
:10084000FC0180819181892B21F460E070E0CB0173
:10085000089564E477E080E090E008958F929F929D
:10086000AF92BF92CF92DF92EF92FF920F931F93BE
:10087000CF93DF93CDB7DEB7CB54D1090FB6F89441
:10088000DEBF0FBECDBF8C017B010E94AA022C9659
:100890009FAF8EAF2C97CE01865B9F4F0E942004A6
:1008A000672B09F09DC080FD9BC0C8010E944102DA
:1008B000873291F4BE016F5B7F4FC8010E945102E5
:1008C0009A838983CE0101960E942004672B09F048
:1008D000BDC180FDBBC1BDC1883204F5823251F378
:1008E000C8010E944102C82EFE0131964F01D12C51
:1008F0005F018C2D0E942702882309F4BCC1FFE30D
:10090000DF1609F4B8C1F8011086D394D401CD9252
:100910004D01C8010E944102C82EEBCF8B3561F515
:10092000D70114968C9114978078806414968C93D8
:10093000149711961C921E9213961C921E92129757
:10094000F8018681882379F1C8010E9441028B3524
:1009500009F073C1D80118961C92C8010E94AA021E
:100960009A838983CE0101960E942004672B09F0A7
:100970006DC180FD6BC13BC08B3709F0B1CFD70192
:1009800014968C9114978078806214968C931497A7
:1009900011961C921E9213961C921E921297F801A9
:1009A0008681811102C085E064C1C8010E944102B4
:1009B0008B3709F042C1D80118961C92C8010E94D9
:1009C000AA0223969FAF8EAF2397CE018F5B9F4FD6
:1009D0000E942004672B09F032C180FD30C117C18D
:1009E0002B968FAD2B972C969FAD2C97BCC1C80131
:1009F0000E9441028D35B9F1D8016D917C91C701FA
:100A00000E94F002BC01892B09F4F7C0F80196811D
:100A100091509683C8010E942E049A838983D8013D
:100A200016968C9116978F5F16968C93CE01019631
:100A30000E942004672B09F009C180FD07C1C8018D
:100A40000E94AA029A838983CE0101960E94200403
:100A5000672B09F0FBC080FDF9C0C8010E9441026C
:100A60008D3509F0CCC0F801108602C1C8010E9482
:100A70004102873209F4D1C0823209F4CEC0D801D4
:100A800014968D909C901597C8010E944102B82E33
:100A9000882309F4CFC08B2D0E942702882309F4F4
:100AA000C3C0F80110860480F581E02DCF010196C6
:100AB000D80115969C938E931497B082C8010E941A
:100AC0004102B82E0E9427028111EBCFD801149663
:100AD000ED91FC911597CF01019615969C938E93FD
:100AE000149710829A828982892809F4A0C080E034
:100AF00090E023969FAF8EAF2397CE018F5B9F4FE1
:100B00000E942004672B09F09AC080FD98C02981BB
:100B10003A81F60184818068848337832683C80103
:100B20000E94AA0223969FAF8EAF2397CE018F5BC0
:100B30009F4F0E942004672B09F081C080FD7FC079
:100B4000C8010E9441028A3309F077C0F80110867B
:100B5000868181508683B601C8010E942E042396A7
:100B60009FAF8EAF2397D80116968C9116978F5F03
:100B700016968C93CE018F5B9F4F0E942004672BAB
:100B800009F05DC080FD5BC0C8010E94AA022396E7
:100B90009FAF8EAF2397CE018F5B9F4F0E942004A3
:100BA000672B09F04CC080FD4AC0C8010E94410279
:100BB0008D3709F458CFC8010E9441028C32E9F503
:100BC000D80118961C92C8010E94AA0223969FAFD2
:100BD0008EAF2397CE018F5B9F4F0E942004672B1F
:100BE00071F580FD2CC0D8016D917C91C7010E94E8
:100BF000F0026C01892B09F039CF83E03AC0C801BB
:100C00000E9441028C32C9F4F8011086F5CEC80169
:100C10000E9441028D3739F726CFBE016F5F7F4FAB
:100C2000C8010E94510265CF82E090E062CF83E06C
:100C300090E05FCF81E090E05CCF82E01AC0229626
:100C40008FAD229723969FAD23978DC089819A817E
:100C50008AC023962EAD3FAD2397D70114968C9171
:100C600014978078856014968C9314972D933C93F9
:100C700080E090E078C0F501ED0DF11D10828981D2
:100C80008437A1F4D70114968C91149780788660EC
:100C900014968C9381E090E0A0E0B0E0F7018083AF
:100CA0009183A283B38390E0F4E012C0863699F476
:100CB000D70114968C9114978078866014968C9343
:100CC000F701108211821282138281E090E0F5E038
:100CD000DF1249C007C08E3639F481E090E024E08D
:100CE000D21241C080E03FC0B501CE018F5B9F4F63
:100CF0000E94D20025964CAD5DAD6EAD7FAD2597BF
:100D00002A968FAD2A978A3061F08C30C1F08830F6
:100D100009F093CFD70114968C911497807888604E
:100D200006C0D70114968C91149780788A60149627
:100D30008C93F701408351836283738399CF299603
:100D40004CAD5DAD6EAD7FAD2997D70114968C91FA
:100D5000149780788C6014968C93F70140835183AC
:100D60006283738385CFC55BDF4F0FB6F894DEBF18
:100D70000FBECDBFDF91CF911F910F91FF90EF90EC
:100D8000DF90CF90BF90AF909F908F9008958EBDD1
:100D900000000DB407FEFDCF8EB50895CF93DF930D
:100DA000EC018E8184608E8360E088810E941E0940
:100DB00084E00E94C7068E810E94C7068E8182FF52
:100DC00008C084E80E94C70680E00E94C7068E83A0
:100DD000F5CF61E08881DF91CF910C941E09FC0171
:100DE000828193810E94CE0681E00895CF93DF93A4
:100DF000EC016F736C834F714D8360E088810E94BA
:100E00001E0982E00E94C7068C810E94C70683E00B
:100E10000E94C7068D810E94C70661E08881DF912C
:100E2000CF910C941E09FC01828193810E94F606E9
:100E300081E00895CF92DF92EF92FF920F931F937C
:100E4000CF93DF936C017A018B01C0E0D0E0CE1527
:100E5000DF0581F0D8016D918D01D601ED91FC91F6
:100E60000190F081E02DC6010995892B11F02196A2
:100E7000EECF7E01C701DF91CF911F910F91FF90BF
:100E8000EF90DF90CF900895089580E090E008956E
:100E9000FC01538D448D252F30E0842F90E0821B80
:100EA000930B541710F0CF9608950197089586E993
:100EB00092E00E94BC0021E0892B09F420E0822FFF
:100EC00008950E94BB10EF92FF920F931F93CF9350
:100ED000DF93EC0181E0888F9B8D8C8D981305C08A
:100EE000E889F989808185FD26C0F62E0B8D10E0FA
:100EF0000F5F1F4F0F731127E02E8C8DE8120CC06F
:100F00000FB607FCFACFE889F989808185FFF5CF14
:100F1000CE010E942E03F1CF8B8DFE01E80FF11D53
:100F2000E35AFF4FF0829FB7F8940B8FEA89FB8951
:100F3000808180620AC09FB7F894EE89FF89608340
:100F4000E889F98980818370806480839FBF81E014
:100F500090E0DF91CF911F910F91FF90EF90089556
:100F6000CF93DF93EC01888D8823C9F0EA89FB8950
:100F7000808185FD05C0A889B9898C9186FD0FC047
:100F80000FB607FCF5CF808185FFF2CFA889B9891C
:100F90008C9185FFEDCFCE010E942E03E7CFDF912C
:100FA000CF9108951F920F920FB60F9211242F9395
:100FB0003F934F935F936F937F938F939F93AF93E1
:100FC000BF93EF93FF9386E992E00E942E03FF9177
:100FD000EF91BF91AF919F918F917F916F915F91B1
:100FE0004F913F912F910F900FBE0F901F9018952A
:100FF0001F920F920FB60F9211242F938F939F93EE
:10100000EF93FF93E091A602F091A7028081E09117
:10101000AC02F091AD0282FD12C090818091AF02CE
:101020008F5F8F732091B002821751F0E091AF0271
:10103000F0E0EA56FD4F958F8093AF0201C08081AA
:10104000FF91EF919F918F912F910F900FBE0F9075
:101050001F9018953FB7F89480915D0390915E03BF
:10106000A0915F03B091600326B5A89B05C02F3FF8
:1010700019F00196A11DB11D3FBFBA2FA92F982FBE
:101080008827820F911DA11DB11DBC01CD0142E039
:10109000660F771F881F991F4A95D1F7089500970B
:1010A00069F0FC0101900020E9F73197AF01481B7E
:1010B000590BBC0186E992E00C941A0780E090E09D
:1010C0000895CF93DF930E944F08EC0180E992E0EE
:1010D0000E944F088C0F9D1FDF91CF91089590E0E3
:1010E000FC01E753FF4F2491FC01EB54FF4F849127
:1010F000882399F090E0880F991FFC01E555FF4F78
:10110000A591B491FC01EF55FF4F859194918FB754
:10111000F894EC91E22BEC938FBF08958F929F92FD
:10112000AF92BF92CF92DF92EF92FF920F931F93F5
:10113000CF93DF93CDB7DEB7A1970FB6F894DEBF9C
:101140000FBECDBF6C01990FEE08FF08F7FE2BC054
:101150006DE286E992E00E9463078C012227332723
:10116000A9012C193D094E095F0919A2CE018196EA
:101170007C019AE0892E912CA12CB12CCA01B901D5
:10118000A50194010E94370F605DF70162937F0112
:10119000211531054105510589F7CF010E944F08FE
:1011A000800F911F1DC0A701960119A28E010F5D2E
:1011B0001F4F8AE0C82ED12CE12CF12CCA01B901B5
:1011C000A70196010E94370F605DF80162938F01BD
:1011D000211531054105510589F7CF010E944F08BE
:1011E000A1960FB6F894DEBF0FBECDBFDF91CF91B1
:1011F0001F910F91FF90EF90DF90CF90BF90AF9035
:101200009F908F9008950F931F93CF93DF938C013E
:10121000C0E0D0E0F801EC0FFD1F6491662341F0BF
:1012200086E992E00E946307892B11F02196F2CFA4
:10123000CE01DF91CF911F910F91089590E0FC01B5
:10124000E357FF4F2491FC01E753FF4F3491FC011A
:10125000EB54FF4FE491EE2309F43CC0222339F113
:10126000233091F038F42130A9F0223001F584B513
:101270008F7D12C0273091F02830A1F02430B9F4CE
:10128000809180008F7D03C0809180008F77809354
:1012900080000DC084B58F7784BD09C08091B000F7
:1012A0008F7703C08091B0008F7D8093B000F0E015
:1012B000EE0FFF1FEF55FF4FA591B4919FB7F89424
:1012C000611104C08C913095382302C0EC913E2B03
:1012D0003C939FBF08959F92AF92BF92CF92DF92AF
:1012E000EF92FF920F931F93CF93DF938C016115C1
:1012F000710509F46AC0FB019081D0E0992331F0B7
:10130000DF5FFB01ED0FF11D9081F8CF922EC42F0E
:101310005B01CD2ED12CC6010E949A0F7C01F501F4
:10132000DC018A2F8E198D1740F4919180EE890F80
:101330008B3508F0892F8D93F4CFD0E0FEE19F9E8E
:10134000C00DD11D112481E0F801868360E0808109
:101350000E941E0984E00E94C706F80186810E944F
:10136000C70685E00E94C7068D2F0E94C70686E04B
:101370000E94C7068C2F0E94C706E701CE018E1976
:101380009F098C159D0544F4B99087E00E94C7061B
:101390008B2D0E94C706F2CF87E00E94C7068FEF11
:1013A0000E94C70661E0F80180810E941E09C70102
:1013B000DF91CF911F910F91FF90EF90DF90CF9031
:1013C000BF90AF909F900C943210DF91CF911F91FE
:1013D0000F91FF90EF90DF90CF90BF90AF909F90D4
:1013E00008958F929F92AF92BF92CF92DF92EF9229
:1013F000FF926B017C010E942A084B015C01C11421
:10140000D104E104F104F1F00E942A08DC01CB01CF
:1014100088199909AA09BB09883E9340A105B1051D
:1014200070F321E0C21AD108E108F10888EE880EB5
:1014300083E0981EA11CB11CC114D104E104F10485
:1014400019F7DDCFFF90EF90DF90CF90BF90AF9076
:101450009F908F9008951F920F920FB60F921124B4
:101460002F933F938F939F93AF93BF938091590393
:1014700090915A03A0915B03B0915C0330915803A3
:1014800023E0230F2D3720F40196A11DB11D05C0C7
:1014900026E8230F0296A11DB11D209358038093C7
:1014A000590390935A03A0935B03B0935C0380911C
:1014B0005D0390915E03A0915F03B091600301967C
:1014C000A11DB11D80935D0390935E03A0935F0304
:1014D000B0936003BF91AF919F918F913F912F91F6
:1014E0000F900FBE0F901F901895CF93DF93CDB73D
:1014F000DEB7C85BD1090FB6F894DEBF0FBECDBF13
:10150000789484B5826084BD84B5816084BD85B5DE
:10151000826085BD85B5816085BD80916E008160EA
:1015200080936E0010928100809181008260809390
:101530008100809181008160809381008091800092
:101540008160809380008091B10084608093B100BD
:101550008091B00081608093B00080917A008460B7
:1015600080937A0080917A00826080937A008091E3
:101570007A00816080937A0080917A0080688093FD
:101580007A001092C100E091A602F091A70282E0D9
:101590008083E091A202F091A3021082E091A40264
:1015A000F091A50280E180831092AE02E091AA0240
:1015B000F091AB0286E08083E091A802F091A9024D
:1015C000808180618083E091A802F091A9028081EE
:1015D00088608083E091A802F091A90280818068F0
:1015E0008083E091A802F091A90280818F7D8083A1
:1015F00081E791E00E94610882EC91E00E9461081D
:101600008AED91E00E9461088AEE91E00E946108F3
:1016100081E791E00E9461088AE092E00E946108FF
:101620001FB7F89480919402811124C0EFEBF0E091
:101630008491E3EDF0E09491E82FF0E0EE0FFF1FCE
:10164000E555FF4FA591B491EC91E92321F461E0B8
:101650008AE00E941E098AE00E946F088CB58061B2
:101660008CBD8CB580648CBD8DE00E946F088BE0D2
:101670000E946F08809194028F5F809394021FBF35
:1016800086E0809335031092360387E48093380315
:1016900086E00E946F0861E086E00E941E0964E611
:1016A00070E080E090E00E94F10960E080913503F5
:1016B0000E941E0980E00E94C70682E480933703DF
:1016C0000E94C70661E0809135030E941E0964EF05
:1016D00071E080E090E00E94F10960E080913503C4
:1016E0000E941E0934E4E32E33E0F32E00E010E004
:1016F0006701D7011D927D01F801EC5BFC4F8081F1
:101700008C7F8260808380E1800F0E94C706F60193
:1017100080810E94C7060F5F1F4F0031110541F7FE
:1017200084E08093370380E00E94C70680913703EE
:101730000E94C70661E0809135030E941E0985E37F
:1017400093E00E94CE064BE161E385E393E00E94C3
:10175000F60680913803807F8E608093380360E0C6
:10176000809135030E941E0981E00E94C706809186
:1017700038030E94C70661E0809135030E941E096C
:101780008091360381111AC080913703806488608C
:101790008093370360E0809135030E941E0980E04A
:1017A0000E94C706809137030E94C70661E08091BE
:1017B00035030E941E0981E0809336038091370330
:1017C00080638093370360E0809135030E941E0997
:1017D00080E00E94C706809137030E94C70661E03F
:1017E000809135030E941E0920E040E067EA71E025
:1017F00085E393E00E946B0921E040E062EC71E038
:1018000085E393E00E946B0922E040E06AED71E01D
:1018100085E393E00E946B0923E040E06AEE71E00B
:1018200085E393E00E946B0924E040E067EA71E001
:1018300085E393E00E946B0968EB7BE080E090E039
:101840000E94F10985E393E00E94CE0688E192E0D0
:101850000E9461088E010F571F4F3801FDE06F0E87
:10186000711C780188E0E80EF11C28019DE2490E08
:10187000511C1801A8E02A0E311C86E992E00E9452
:10188000BC00181619060CF0A0C086E992E00E9470
:101890009A00D82E80919502BAE0E1E0F0E0EC0FDA
:1018A000FD1FE80FF11DDB1659F0D0828F5F87FD19
:1018B00003C080939502E1CFEFE7E0939502DDCF7F
:1018C0001082109295028FE192E00E944F08CE01A3
:1018D00001960E946108D80111967C926E9213962F
:1018E0007C926E92129715965C924E921497179670
:1018F0005C924E9216971C968C911C9780781C9641
:101900008C93C255DF4F19830883CE5AD040E1E053
:10191000F0E0EC0FFD1FC055DF4FF983E883C05B9B
:10192000D040CE54DF4FF983E883C25BD040CC5423
:10193000DF4FD882C45BD040CA54DF4F1882C65BE9
:10194000D040B101CE0182559F4F0E942E04C95450
:10195000DF4F99838883C75BD040CE0189549F4F66
:101960000E942004672BD9F480FD19C0CB54DF4FAF
:101970008881C55BD040882391F0D8011C968C915A
:10198000982F907661F48F778450823040F0E2E0B7
:10199000F0E0C954DF4FF983E883C75BD040C954F6
:1019A000DF4F88819981C75BD040C255DF4F998353
:1019B0008883CE5AD040CE0182559F4F0E9420048A
:1019C000672B31F480FD04C01DC00E94C8004DCFBC
:1019D00082E790E00E940309C255DF4F8881998118
:1019E000CE5AD0408630910550F4880F991FFC01E3
:1019F000EA5CFE4F808191810E9461083ECF8DE6B6
:101A000091E0FACF64E472E0C7010E94D003FC01C8
:101A1000892B41F094819F779450923018F4C080C4
:101A2000D18002C0C12CD12CB6018AE292E00E9482
:101A3000C010892B09F06AC060E372E0C7010E9400
:101A4000D003009709F462C0DC0114968C918F7763
:101A50008450823008F05AC065E372E0C7010E94EA
:101A6000D0030E94FF03882309F450C069E772E0A5
:101A7000C7010E94D0030E94FF03882309F446C0D7
:101A800060E372E0C7010E94D003FC01892B41F0A2
:101A900094819F779450923018F4C080D18002C016
:101AA000C12CD12C65E372E0C7010E94D0030E94D3
:101AB00050035C0169E772E0C7010E94D0030E94F5
:101AC00050034C0188E690E00E940309C5010E9482
:101AD0008E0887E392E00E944F08C4010E948E089E
:101AE00089E392E00E944F08C6010E94610880913C
:101AF000330390913403DC01ED91FC910190F0816E
:101B0000E02D9601A401B5010995B7CEB6018CE48C
:101B100092E00E94C010892B59F480913303909178
:101B20003403DC01ED91FC910280F381E02D0995F5
:101B3000B6018DE392E00E94C010892B09F09DCE82
:101B400065E372E0C7010E94D0030E9450036C015C
:101B500069E772E0C7010E94D0030E945003A09180
:101B60003303B0913403ED91FC9111970480F5811A
:101B7000E02DAC01B601CD0109957FCEE6E9F2E09A
:101B80001382128288EE93E0A0E0B0E08483958314
:101B9000A683B78386E491E09183808385EC90E00F
:101BA0009587848784EC90E09787868780EC90E027
:101BB000918B808B81EC90E0938B828B82EC90E018
:101BC000958B848B86EC90E0978B868B118E128E92
:101BD000138E148EE1E6F3E088E591E09183808333
:101BE00085E393E093838283F0933403E09333039C
:101BF00008950E943B0E08F481E00895E89409C01E
:101C000097FB3EF490958095709561957F4F8F4F2F
:101C10009F4F9923A9F0F92F96E9BB279395F69545
:101C2000879577956795B795F111F8CFFAF4BB0FC3
:101C300011F460FF1BC06F5F7F4F8F4F9F4F16C027
:101C4000882311F096E911C0772321F09EE8872FB1
:101C5000762F05C0662371F096E8862F70E060E06D
:101C60002AF09A95660F771F881FDAF7880F9695E6
:101C7000879597F90895990F0008550FAA0BE0E88A
:101C8000FEEF16161706E807F907C0F0121613063E
:101C9000E407F50798F0621B730B840B950B39F47E
:101CA0000A2661F0232B242B252B21F408950A26E4
:101CB00009F4A140A6958FEF811D811D08950E9412
:101CC000720E0C94E30E0E94D50E38F00E94DC0ECA
:101CD00020F0952311F00C94CC0E0C94D20E11240C
:101CE0000C94170F0E94F40E70F3959FC1F3950F9B
:101CF00050E0551F629FF001729FBB27F00DB11D90
:101D0000639FAA27F00DB11DAA1F649F6627B00D1F
:101D1000A11D661F829F2227B00DA11D621F739F08
:101D2000B00DA11D621F839FA00D611D221F749F16
:101D30003327A00D611D231F849F600D211D822F5D
:101D4000762F6A2F11249F5750409AF0F1F0882384
:101D50004AF0EE0FFF1FBB1F661F771F881F9150B1
:101D60005040A9F79E3F510580F00C94CC0E0C9486
:101D7000170F5F3FE4F3983ED4F386957795679508
:101D8000B795F795E7959F5FC1F7FE2B880F911DDB
:101D90009695879597F9089597F99F6780E870E081
:101DA00060E008959FEF80EC089500240A941616D1
:101DB000170618060906089500240A941216130639
:101DC000140605060895092E0394000C11F48823C7
:101DD00052F0BB0F40F4BF2B11F460FF04C06F5FE3
:101DE0007F4F8F4F9F4F089557FD9058440F551FB9
:101DF00059F05F3F71F04795880F97FB991F61F08D
:101E00009F3F79F087950895121613061406551F03
:101E1000F2CF4695F1DF08C0161617061806991F6F
:101E2000F1CF86957105610508940895E894BB2764
:101E300066277727CB0197F908950E94280FA59F61
:101E4000900DB49F900DA49F800D911D11240895B5
:101E5000A29FB001B39FC001A39F700D811D1124EB
:101E6000911DB29F700D811D1124911D0895A1E255
:101E70001A2EAA1BBB1BFD010DC0AA1FBB1FEE1F04
:101E8000FF1FA217B307E407F50720F0A21BB30B4F
:101E9000E40BF50B661F771F881F991F1A9469F7CB
:101EA00060957095809590959B01AC01BD01CF0127
:101EB0000895EE0FFF1F0590F491E02D09940E9404
:101EC000660F6894B1110C94170F08950E94FC0ED0
:101ED00088F09F5798F0B92F9927B751B0F0E1F0EB
:101EE000660F771F881F991F1AF0BA95C9F714C09B
:101EF000B13091F00E94160FB1E008950C94160FC6
:101F0000672F782F8827B85F39F0B93FCCF38695D3
:101F100077956795B395D9F73EF490958095709530
:101F200061957F4F8F4F9F4F08950E943B0E08F49D
:101F30008FEF08950F931F93CF93DF938230910516
:101F400010F482E090E0E0916703F091680320E0F4
:101F500030E0A0E0B0E0309719F14081518102817A
:101F6000138148175907C8F08417950769F410972B
:101F700031F012960C93129713961C9327C000937E
:101F800067031093680322C02115310519F0421729
:101F9000530718F49A01BD01EF01DF01F801DBCF0F
:101FA00021153105F9F0281B390B2430310580F457
:101FB0008A819B816115710521F0FB0193838283E6
:101FC00004C09093680380936703FE01329644C077
:101FD000FE01E20FF31F819391932250310939835F
:101FE00028833AC02091650330916603232B41F486
:101FF0002091020130910301309366032093650321
:1020000020910001309101012115310541F42DB7D6
:102010003EB74091040150910501241B350BE0911E
:102020006503F0916603E217F307A0F42E1B3F0B44
:102030002817390778F0AC014E5F5F4F241735073A
:1020400048F04E0F5F1F50936603409365038193E2
:10205000919302C0E0E0F0E0CF01DF91CF911F91BA
:102060000F910895CF93DF93009709F481C0FC018D
:10207000329713821282A0916703B0916803109780
:1020800081F420813181820F931F2091650330916B
:1020900066032817390751F5F0936603E09365034B
:1020A00067C0ED0120E030E0CE17DF0740F44A8141
:1020B0005B819E0141155105F1F0EA01F5CFD38313
:1020C000C28340815181840F951FC817D90759F4E5
:1020D00088819981840F951F0296918380838A81DC
:1020E0009B81938382832115310529F4F093680342
:1020F000E09367033DC0E901FB83EA83499159916D
:10210000C40FD51FEC17FD0761F480819181840F06
:10211000951F0296E90199838883828193819B832D
:102120008A83E0E0F0E012968D919C9113970097DE
:1021300019F0FD01DC01F7CF8D919C9111979D0164
:102140002E5F3F4F820F931F2091650330916603EE
:102150002817390769F4309729F410926803109210
:10216000670302C013821282B0936603A0936503D3
:10217000DF91CF91089581E090E0F8940C94C9101C
:10218000FB01DC018D91019080190110D9F3990BAD
:062190000895F894FFCF52
:10219600000069032000CDCCCC3D0AD7233C17B7FD
:1021A600D13877CC2B329595E6241FB14F0A000023
:1021B60020410000C84200401C4620BCBE4CCA1B41
:1021C6000E5AAEC59D7452025502650272027B021A
:1021D60088020000000063071A074807B007BC0022
:1021E6009A00AE00000000002303EF061307222228
:1021F6005C5C6208660C6E0A720D7409003F3F3F14
:10220600003D3D3D3D3D3D3D3D3D3D3D3D3D3D3D35
:102216003D3D3D3D3D3D3D3D3D3D3D3D3D3D3D3DE8
:102226003D3D3D3D3D3D3D3D3D3D3D3D3D3D3D3DD8
:102236003D3D3D3D3D3D3D3D3D3D3D3D3D3D3D3DC8
:102246003D3D3D3D3D3D3D3D3D3D3D3D3D3D3D3DB8
:102256003D004669726D776172653A204D696E6917
:102266006D4F53442D4A534F4E0056657273696F36
:102276006E3A2020302E312E31004275696C743A48
:10228600202020204F637420203820323031392C12
:102296002031333A33383A343800496E697469610B
:1022A6006C697A652E2E2E0052656164792100488C
:1022B600616E646C696E673A2000777269746500B6
:1022C600746578740078002C00293A20006F6666E1
:1022D60073657400636F6D6D616E6400636C656138
:1022E60072004F6B00496E636F6D706C6574654963
:1022F6006E70757400496E76616C6964496E7075AE
:1023060074004E6F4D656D6F7279004E6F74537524
:1023160070706F7274656400546F6F446565700009
:042326000D0A00009C
:00000001FF
